:100000000C9434000C9451000C9451000C94510049
:100010000C9451000C9451000C9451000C9451001C
:100020000C9451000C9451000C9451000C9451000C
:100030000C9451000C9451000C9451000C945100FC
:100040000C9451000C9451000C9451000C945100EC
:100050000C9451000C9451000C9451000C945100DC
:100060000C9451000C94510011241FBECFEFD4E02A
:10007000DEBFCDBF11E0A0E0B1E0E2E7FDE002C0ED
:1000800005900D92A830B107D9F711E0A8E0B1E0D2
:1000900001C01D92A830B107E1F70E9458000C94EE
:1000A000B8060C9400008EBD0DB407FEFDCF089578
:1000B000CFEFD4E0DEBFCDBF519A509A559A3A9A0D
:1000C000259A239A229A2A9A3A9A299A5E9A219AEA
:1000D000569A5A9A5B9A83E58CBD83E680937C009E
:1000E00087E880937A0088E080937E0083B7816000
:1000F00083BFEE24FE2CCFE788E893E10197F1F768
:10010000E7FE08C08E2D992788779070892B11F40F
:100110005D9A01C05D9880917A00806480937A0036
:1001200080917A0086FDFCCF00917900F01610F4E2
:10013000429A01C04298802F99278F199109AA27C6
:1001400097FDA095BA2FBC01CD010E94F603DC01FA
:10015000CB019C01AD016AE979E989ED9FE30E9439
:10016000A502DC01CB0120E030E04CED52E4BC0103
:10017000CD010E943F02DC01CB01BC01CD010E94F8
:10018000F100DC01CB01813C08F080ECC81708F4D9
:10019000CF5F8C1708F4C150299814E1812F8A95FC
:1001A000F1F78C2F0E9453008C2F0E9453008C2F4C
:1001B0000E9453008C2F0E945300812F8A95F1F7E3
:1001C000299A4B9904C0F01608F4F02E599A4A99CE
:1001D00004C0FF24589A4A9BFDCF59985898E3943D
:1001E0008BCFEF92FF920F931F937B018C0120E046
:1001F00030E040E05FE40E94C00388239CF020E0F0
:1002000030E040E05FECC801B7010E943F02DC0132
:10021000CB01BC01CD010E945A0460507040804067
:10022000904804C0C801B7010E945A041F910F9161
:10023000FF90EF900895A0E0B0E0E1E2F1E00C94CF
:1002400081068C017B015A01DC018C91823058F0CF
:10025000FB019081923010F4A7010BC1843029F486
:10026000943009F4A6C0A80104C19430A9F39230D7
:1002700009F4A9C0823081F3F801C280D380FB0168
:1002800062817381F8012481358146815781F701AC
:100290006480758086809780C601861B970B97FDCA
:1002A000D8C080970CF46CC06C157D050CF0ADC007
:1002B000662477244301F8016181F7018181681781
:1002C00009F499C0662309F491C0621A730A840A7A
:1002D000950AA401930157FDC0C0F5011182B60132
:1002E00019012A0179018A0139014A01089461083A
:1002F000710881089108FFEF6F16FFEF7F06FFEF8F
:100300008F06FFE39F06F0F4A8019701220F331F29
:10031000441F551F19012A01B601615070406B013D
:1003200079018A0139014A0108946108710881083C
:1003300091088FEF68168FEF78068FEF88068FE3AE
:10034000980610F383E0D5018C9357FC64C0F50147
:10035000248335834683578373836283A50189C0D1
:100360006F5F7F4FD401C30181709070A070B07037
:100370009694879477946794682A792A8A2A9B2A84
:100380006C157D056CF311C00894C11CD11CDA01F9
:10039000C90181709070A070B070569547953795DF
:1003A0002795282B392B4A2B5B2BC616D70664F3CF
:1003B00082CFF8019181FB018181981709F453CF15
:1003C00040E051E056C0823009F04DCFDA01F8012B
:1003D00088E001900D928150E1F7F8018181F701E9
:1003E00091818923F5018183A50143C0261937092D
:1003F0004809590970CFF5016183B601260D371DF3
:10040000481D591D19012A019DCF6B0120E030E0E4
:1004100040E050E050CFD201C101B695A795979525
:10042000879521E030E040E050E022223322442250
:100430005522282A392A4A2A5B2AF5012482358244
:10044000468257820894C11CD11CD382C282A50166
:1004500010C0909581959F4F24CF81E0F501818355
:10046000B60150954095309521953F4F4F4F5F4FC6
:1004700037CFCA01E2E1CDB7DEB70C949D06A0E20A
:10048000B0E0E5E4F2E00C948F06DC01CB01898F4B
:100490009A8FAB8FBC8F2D8F3E8F4F8F58A3BE018D
:1004A0006F5F7F4FCE0149960E9494058E01075FD2
:1004B0001F4FB801CE014D960E949405AE014F5ECC
:1004C0005F4FB801CE0101960E941B010E94AC044F
:1004D000DC01CB01BC01CD01E4E0A0960C94AB069D
:1004E000A0E2B0E0E6E7F2E00C948F06DC01CB017D
:1004F000898F9A8FAB8FBC8F2D8F3E8F4F8F58A3D4
:10050000BE016F5F7F4FCE0149960E9494058E0118
:10051000075F1F4FB801CE014D960E9494058A8552
:1005200091E089278A87AE014F5E5F4FB801CE0107
:1005300001960E941B010E94AC04DC01CB01BC01AE
:10054000CD01E4E0A0960C94AB06A0E2B0E0EBEAAB
:10055000F2E00C948106DC01CB01898F9A8FAB8F7E
:10056000BC8F2D8F3E8F4F8F58A3BE016F5F7F4F83
:10057000CE0149960E94940569E070E06C0F7D1FE2
:10058000CE014D960E949405FE0131966624772493
:100590004301130124018981823098F099859230BA
:1005A00058F420E091818A85981321E02A8769E038
:1005B00070E06C0F7D1FD9C0843059F4923009F47B
:1005C0005BC020E091818A85981321E02183BF01DF
:1005D000CCC0943009F44DC0823099F3923009F3C5
:1005E000ED80FE800F8118852D853E854F855889C9
:1005F000640153016FE170E00CC0220F331F441FF0
:10060000551F16950795F794E7946150704077FD54
:1006100036C0D801C70181709070A070B070892B6E
:10062000C9F080E090E0220E331E441E551E2216B3
:1006300033064406550610F481E090E0AA2797FDA2
:10064000A095BA2F8A0D9B1DAC1DBD1D680E791E8D
:100650008A1E9B1EAA0CBB1CCC1CDD1C57FFCDCFD9
:1006600081E090E0A0E0B0E0A82AB92ACA2ADB2AFB
:10067000C4CF823009F095CF60E071E076C022816E
:1006800033818B859C85280F391F2E5F3F4FA90131
:1006900060E091818A85981361E06A8B97FE0FC0B4
:1006A0002FC0CA010197AC019C01660C771C881C05
:1006B000991C57FC41C0220C331C441C551C90E073
:1006C000691690E0790690E0890690E4990648F36F
:1006D0003C8B2B8BD401C3018F779070A070B070CE
:1006E00080349105A105B10581F16D8A7E8A8F8ADA
:1006F000988E83E0898B61E170E06C0F7D1F35C0BF
:100700002F5F3F4FA901D401C30181709070A07089
:10071000B070892B61F0569447943794279480E009
:1007200090E0A0E0B0E8282A392A4A2A5B2A969469
:10073000879477946794C3CF81E090E0A0E0B0E025
:10074000682A792A8A2A9B2AB6CF67FC05C0211419
:1007500031044104510449F280E490E0A0E0B0E0AB
:10076000680E791E8A1E9B1EC0CFCB010E94AC046E
:10077000DC01CB01BC01CD01E2E1A0960C949D0609
:10078000A8E1B0E0E6ECF3E00C948F06DC01CB01CD
:10079000898B9A8BAB8BBC8B2D8B3E8B4F8B588F61
:1007A000BE016F5F7F4FCE0141960E9494058E017E
:1007B000075F1F4FB801CE0145960E9494058981BD
:1007C000823018F08985823018F42FEF3FEF09C08E
:1007D000B801CE0101960E940E06282F332727FD6F
:1007E0003095C901E4E068960C94AB06A8E0B0E04F
:1007F000ECEFF3E00C948D069B01AC017B018C01C6
:10080000EE2417FDE394FF2400271127EA82211527
:1008100031054105510539F482E08983CE01019605
:100820000E94AC0443C083E089836EE170E0CB0199
:10083000EE2031F579018A01A80197012030E0E02E
:100840003E07E0E04E07E0E45E0798F479018A0194
:10085000EE0CFF1C001F111F0197BC01A80197019E
:10086000E0E0EE16E0E0FE06E0E00E07E0E41E0742
:1008700068F3ED82FE820F8318877C836B83CECF73
:100880002030E0E03E07E0E04E07E0E85E0741F0A0
:10089000EE24FF248701E21AF30A040B150BCCCFD8
:1008A0007C836B8360E070E080E09FECE6E028965C
:1008B0000C94A906ACE0B0E0E0E6F4E00C949106FC
:1008C000DC01CB0189879A87AB87BC87BE016F5F4C
:1008D0007F4FCE0109960E9494058981823011F0E4
:1008E000823028F460E070E080E090E031C0843035
:1008F00039F02B813C8137FDF5CF2F3131056CF07C
:100900008A81882329F060E070E080E090E820C0D0
:100910006FEF7FEF8FEF9FE71BC08EE190E0821BB0
:10092000930B2D813E814F81588504C05695479584
:10093000379527958A95D2F78A81882339F0509583
:100940004095309521953F4F4F4F5F4FCA01B901F8
:10095000E2E02C960C94AD06A0E0B0E0E2EBF4E00F
:100960000C948706882499245401DC01FC0124811D
:100970003581468157818181082F112760E070E021
:100980008C91823020F46FEF70E04061A4C084301D
:1009900009F464C0823009F463C0211531054105B2
:1009A000510509F498C0FD0182819381FFEF8238DF
:1009B0009F070CF050C0A2E8EA2EAFEFFA2EE81A1B
:1009C000F90A8AE1E816F1040CF06BC06B0181E0D2
:1009D00090E0A0E0B0E00E2C04C0880F991FAA1F81
:1009E000BB1F0A94D2F70197A109B109822393236F
:1009F000A423B5230097A105B10519F0F1E0CF2E8E
:100A0000D12C04C05695479537952795EA94D2F78F
:100A1000C601AA2797FDA095BA2F282B392B4A2B60
:100A20005B2BDA01C9018F779070A070B0708034B1
:100A30009105A105B105D1F1215C3F4F4F4F5F4FAB
:100A40002030E0E03E07E0E04E07E0E45E0708F11A
:100A500061E070E01EC0803891053CF06FEF70E0FF
:100A600020E030E040E050E036C0BC0161587F4FEC
:100A7000DA01C9018F779070A070B0708034910551
:100A8000A105B105D1F0215C3F4F4F4F5F4F57FD9E
:100A90001BC097E056954795379527959A95D1F7BE
:100AA0001AC020E030E040E050E0BBCF27FFC8CFC5
:100AB000205C3F4F4F4F5F4FC3CF27FFE8CF205CF5
:100AC0003F4F4F4F5F4FE3CF56954795379527954B
:100AD0006F5F7F4FDECF822E932E942F9F778A2DCC
:100AE0008078A82EA92A962F9795992797958A2DD1
:100AF0008F77A82EA92A76956795962F9F778B2DAD
:100B00008078B82EB92A902F9795992797958B2D95
:100B10008F77B82EB92AD501C401BC01CD01ECE014
:100B2000CDB7DEB70C94A306CF93DF93FC01DB01B6
:100B3000408151812281622F6F7770E0221F22272E
:100B4000221F9381892F880F822B282F3327991FEB
:100B50009927991FED0199832115310541F441151C
:100B6000510561057105E1F482E08C9354C02F3F7B
:100B7000310509F441C02F573040FD0133832283F2
:100B800083E08C9387E0440F551F661F771F8A957B
:100B9000D1F77064ED014C835D836E837F833BC02E
:100BA00022E83FEFF901C7E0440F551F661F771F8A
:100BB000CA95D1F783E08C93403080E0580780E0FD
:100BC000680780E4780778F4440F551F661F771F85
:100BD00021503040F9014030C0E05C07C0E06C07B4
:100BE000C0E47C0788F3ED01FB83EA83FD014483C5
:100BF0005583668377830FC04115510561057105E3
:100C000019F484E08C9307C064FF03C081E08C93E7
:100C1000C1CF1C92BFCFDF91CF9108950F931F9347
:100C2000CF93DF93FC01DB018081823018F09C912F
:100C3000923018F461E070E05EC08430C1F084301E
:100C400001F1943009F447C0823009F44BC082307E
:100C500009F44EC09230A9F04181ED018981481715
:100C6000B9F0442389F08FEF9FEFBC0144C094306A
:100C700031F7EB018981682F77278181681B710922
:100C80003AC08181882379F781E090E0BC0133C0CC
:100C900022813381ED018A819B81821793070CF3B6
:100CA000281739079CF00481158126813781FD01C1
:100CB0006481758186819781601771078207930728
:100CC00080F2061717072807390778F4442359F2EA
:100CD00081E090E0DBCFFD018181882321F281E07A
:100CE00090E0D4CF923009F0B2CF60E070E003C062
:100CF000ED018981F2CFCB01DF91CF911F910F914F
:100D000008952F923F924F925F926F927F928F92AF
:100D10009F92AF92BF92CF92DF92EF92FF920F938A
:100D20001F93CF93DF93CDB7DEB7CA1BDB0B0FB694
:100D3000F894DEBF0FBECDBF09942A883988488851
:100D40005F846E847D848C849B84AA84B984C884E7
:100D5000DF80EE80FD800C811B81AA81B981CE0FDE
:100D6000D11D0FB6F894DEBF0FBECDBFED010895C3
:020D7000FFCFB3
:080D7200000000000000000079
:00000001FF
